:100000000C9474010C9491010C9491010C94910145
:100010000C9491010C9491010C9491010C94910118
:100020000C9491010C9491010C9491010C94910108
:100030000C9491010C9491010C9491010C949101F8
:100040000C9491010C9491010C9491010C949101E8
:100050000C9491010C94F4060C9491010C94910170
:100060000C9491010C949101808183848687898A04
:100070008C8E8F9192949597989A9B9D9EA0A2A307
:10008000A5A6A7A9AAACADAFB0B2B3B5B6B7B9BA79
:10009000BCBDBEC0C1C2C4C5C6C8C9CACBCDCECF07
:1000A000D0D2D3D4D5D6D7D9DADBDCDDDEDFE0E1C0
:1000B000E2E3E4E5E6E7E8E9EAEAEBECEDEEEEEFB1
:1000C000F0F1F1F2F3F3F4F5F5F6F6F7F8F8F9F9E3
:1000D000FAFAFAFBFBFCFCFCFDFDFDFDFEFEFEFE5C
:1000E000FEFFFFFFFFFFFFFF0000891112239B327D
:1000F0002446AD573665BF74488CC19D5AAFD3BEF8
:100100006CCAE5DB7EE9F7F88110080193331A2207
:10011000A5562C47B7753E64C99C408DDBBF52AED7
:10012000EDDA64CBFFF976E802218B3010029913E7
:100130002667AF763444BD554AADC3BC588ED19FB7
:100140006EEBE7FA7CC8F5D983310A2091121803C7
:10015000A7772E66B5543C45CBBD42ACD99E508F97
:10016000EFFB66EAFDD874C904428D5316619F7097
:100170002004A9153227BB364CCEC5DF5EEDD7FC77
:100180006888E1997AABF3BA85520C4397711E6087
:10019000A1142805B3373A26CDDE44CFDFFD56EC57
:1001A000E9986089FBBB72AA06638F7214409D5167
:1001B0002225AB343006B9174EEFC7FE5CCCD5DD37
:1001C0006AA9E3B8788AF19B87730E6295501C4147
:1001D000A3352A24B1163807CFFF46EEDDDC54CD17
:1001E000EBB962A8F99A708B088481951AA793B627
:1001F0002CC2A5D33EE1B7F04008C919522BDB3A17
:10020000644EED5F766DFF7C899400859BB712A6E6
:10021000ADD224C3BFF136E0C1184809D33B5A2AF6
:10022000E55E6C4FF77D7E6C0AA583B418869197C6
:100230002EE3A7F23CC0B5D14229CB38500AD91BD6
:10024000666FEF7E744CFD5D8BB502A499961087A6
:10025000AFF326E2BDD034C1C3394A28D11A580BB6
:10026000E77F6E6EF55C7C4D0CC685D71EE597F476
:100270002880A1913AA3B3B2444ACD5B5669DF7896
:10028000600CE91D722FFB3E8DD604C79FF516E466
:10029000A9902081BBB332A2C55A4C4BD7795E6876
:1002A000E11C680DF33F7A2E0EE787F61CC495D546
:1002B0002AA1A3B03882B193466BCF7A5448DD5956
:1002C000622DEB3C700EF91F8FF706E69DD414C526
:1002D000ABB122A0B9923083C77B4E6AD5585C4936
:1002E000E33D6A2CF11E780F11241FBECFEFD8E03A
:1002F000DEBFCDBF11E0A0E0B1E0EAE6F7E102C069
:1003000005900D92A231B107D9F718E0A2E1B1E052
:1003100001C01D92A434B107E1F70E946E0A0C944B
:10032000B30B0C9400000C94C40878948CE294E015
:100330000E94100323E931E04CE254E0BA018CE062
:1003400095E00E948D078EEF94E00E94C701EEE3D6
:10035000F8E08EEF94E09383828391838083AC01F5
:100360006CE274E08CE095E00C94B5089091C000CC
:1003700095FFFCCF8093C60081E090E008958091C6
:10038000C00087FFFCCF8091C60090E00895CF9316
:10039000DF93CDB7DEB72E970FB6F894DEBF0FBE52
:1003A000CDBFDC018EE0FD01982F11929A95E9F7FF
:1003B0001092C50097E69093C400E0ECF0E09081C5
:1003C0009D7F908396E09093C20098E19093C10046
:1003D0009E012F5F3F4FF90111928A95E9F783E063
:1003E0008C8386EB91E09A8789878FEB91E09C87DD
:1003F0008B879EE0F90101900D929A95E1F72E9678
:100400000FB6F894DEBF0FBECDBFDF91CF91089538
:10041000811106C08091C000881F8827881F089519
:1004200080E008958091C00087FF03C08091C600DE
:1004300008958FEF08950F931F93CF93DF93182F95
:10044000C0913308D0913408FE01E659FF4F8081F6
:10045000811126C080E490E098A38F8F1E8E1D8EA0
:100460001C8E01E0008331960083299A20910901B6
:1004700030910A0140910B0150910C01A0EBB4E0C6
:100480000E948D0A6056704F8F4F9F4F20E43FE1CE
:1004900040E050E00E94980A3D8B2C8B00931301A2
:1004A0000FB7F894209105013091060140910701A2
:1004B00050910801A0EBB4E00E948D0A6056704F85
:1004C0008F4F9F4F20E43FE140E050E00E94980AA8
:1004D0003F8B2E8B0FBFE0913308F09134084FB75C
:1004E000F89426A137A182A193A12817390739F4DE
:1004F00020A531A584A195A12817390779F060A519
:1005000071A526A137A12150310991E080E0621741
:10051000730709F090E0292F382F02C021E030E066
:100520004FBF232BC1F6E0913308F09134082FB769
:10053000F894A0A5B1A51C9340A551A584A195A1AF
:100540004817590719F482A193A103C080A591A56A
:10055000019691A780A72FBF81E090E0DF91CF9116
:100560001F910F910895E0913308F09134084FB72F
:10057000F894E758FF4F24813581868197814FBFDA
:1005800028173907E9F0E0913308F09134089FB754
:10059000F894E758FF4FA481B58122813381A217D7
:1005A000B30719F42081318105C0A481B5819D0173
:1005B0002F5F3F4F358324838C919FBF90E0089538
:1005C0008FEF9FEF0895109212010895109212017B
:1005D0001092800089E18093810081E896E09093F9
:1005E00087008093860080911201882321F080E4A7
:1005F00080937C0002C010927C00389840988091D3
:100600007E00816080937E0087E080937B008CEE8B
:1006100080937A008AB1886F8AB9219A229A0895C4
:100620000F931F93CF93DF93CDB7DEB72E970FB6FF
:10063000F894DEBF0FBECDBF8C018EECD8011D92A9
:100640008A95E9F7109334080093330880E490E02A
:10065000F80190A3878F11A2C8018C589F4FE459CD
:10066000FF4F918380839783868395838483049649
:10067000938382830996D801A758BF4F11969C9304
:100680008E9317969C938E93169715969C938E93A4
:100690001497CF9613969C938E931297865991092F
:1006A000D80193969C938E93929799969C938E9350
:1006B000989797969C938E939697CF9695969C93A2
:1006C0008E93949784E090E0A681B7811C92468136
:1006D0005781228133814217530719F420813181D8
:1006E00004C0268137812F5F3F4F378326830197D0
:1006F00059F70E94E6028EE0FE013196DF01982F45
:100700001D929A95E9F793E09C832BE132E03A87BA
:10071000298723EB32E03C872B87D80101900D928B
:100720008A95E1F72E960FB6F894DEBF0FBECDBFC7
:10073000DF91CF911F910F9108950F931F93CF9346
:10074000DF93E0913308F091340820A531A537A359
:1007500026A3EC018C01060F171FC017D10731F03B
:1007600060E070E089910E941B02F7CFDF91CF918A
:100770001F910F910895DC0158968C915897811123
:10078000F8C05A968C915A978111AEC096964D91A9
:100790005C91979798962D913C91999742175307A2
:1007A00079F456962D913C915797232B49F410924A
:1007B0001301FD01E659FF4F1082A559BF4F68C0D4
:1007C0005B969C915B97911103C05C961C925C9721
:1007D00091E05B969C935B9754962D913C91559735
:1007E00021153105B9F596964D915C91979798969C
:1007F0002D913C9199974217530779F4FD01E559E2
:10080000FF4F108256962D913C91579721503109F8
:1008100057963C932E93569723C09696ED91FC9154
:10082000979794962D913C919597E217F30729F4A9
:1008300092962D913C91939707C09696ED91FC91DD
:1008400097979F012F5F3F4F97963C932E939697D4
:10085000908107C02150310955963C932E935497AF
:100860009EE759969C93599759969C9159979B311D
:1008700089F596964D915C91979798962D913C911C
:1008800099974217530739F410921301A659BF4F95
:100890001C92299808959696ED91FC9197979496BD
:1008A0008D919C919597E817F90729F492968D916F
:1008B0009C91939706C09696ED91FC919797CF01E6
:1008C000019697969C938E939697808159968C93D8
:1008D000599706C09E57923018F45B961C925B970E
:1008E00081E05A968C935A975B968C915B975F96B2
:1008F0002D913C9190978823A9F05C968C915C9700
:10090000853080F05C961C925C972034310519F09C
:1009100080E490E002C085E790E090969C938E93EF
:100920005F9723C05A968C915A9759969C915997E4
:10093000982341F05C969C915C979F5F5C969C939A
:100940005C970FC05C961C925C972034310519F0BF
:1009500020E430E002C025E730E090963C932E93EF
:100960005F97880F5A968C935A9788E058968C9385
:1009700058975F96ED91FC9190975D968D919C9123
:100980005E97E80FF91F9F0131705E963C932E939E
:100990005D9758968C915897815058968C93FF2765
:1009A000E038F10530F08FEF90E0AC014E1B5F0BAB
:1009B000FA01E859FF4F84912F3F310511F008F0FB
:1009C00080950895EF92FF920F931F93CF93DF933B
:1009D000FC018C010D531F4FD8014D915C91119773
:1009E000129711965C934E93A555B10914968D916B
:1009F0009C91159712962D913C911397821793070E
:100A000021F42D913C91119707C014968D919C91E2
:100A100015979C012F5F3F4F15963C932E9314978B
:100A2000EC012881260290011124C9019595879532
:100A300095958795E801998388837F01D7ECED0E22
:100A4000F11CE701288139818F010B531F4FE80109
:100A500039832883840F951F35952795820F931F1F
:100A6000E70199838883AF0147535F4F21E0181650
:100A700019060CF420E0EA018881880F822B888314
:100A800016968D919C911797EC01688316962D917F
:100A90003C91179712968D919C91139728173907BF
:100AA00021F48D919C91119705C016968D919C9182
:100AB0001797019617969C938E931697DA018C914F
:100AC000982F9695969589278370DF01A653BF4F7F
:100AD000833049F48C91803214F48F5F01C08150CF
:100AE0008C9311A203C081A18F5F81A38C91885F39
:100AF000803414F48C936BC18F738C93DF01A553F6
:100B0000BF4F8C91880F8C93EA01988197702BEFDF
:100B1000290F233010F0933011F481608C938C9165
:100B2000982F96958927809581709685990F892BA6
:100B300086878E3709F052C0DF01A758BF4F149641
:100B40002D913C9115978D919C91119728173907FC
:100B500059F416962D913C91179712968D919C9170
:100B6000139728173907B1F116962D913C911797D5
:100B700014968D919C91159701972817390751F17B
:100B80001696CD91DC9117978EE7888316962D9156
:100B90003C91179712968D919C91139728173907BE
:100BA00021F48D919C91119705C016968D919C9181
:100BB0001797019617969C938E93169791E0918BB9
:100BC0008389863020F4128A8F5F838B01C0928BD9
:100BD00081E0BFC0118A128A138ABAC08F778F371B
:100BE00011F4118A09C08289882311F02A9A01C060
:100BF0002A988189811103C0128A138AE8C08685E8
:100C0000982F9F739E3309F4E2C080FF03C0808950
:100C10008068808B97859F5F97878089983008F4DC
:100C20009DC0DF01A758BF4F92E8980F923018F08F
:100C30008B3109F046C014962D913C9115978D91FA
:100C40009C9111972817390759F416962D913C91CC
:100C5000179712968D919C9113972817390759F180
:100C600016962D913C91179714968D919C911597FE
:100C7000019728173907F9F01696CD91DC9117974F
:100C80008BE1888316962D913C91179712968D9142
:100C90009C9113972817390721F48D919C911197F6
:100CA00005C016968D919C911797019617969C9367
:100CB0008E93169706C0118A128A138A2A9880E0AA
:100CC00001C081E014964D915C9115972D913C9156
:100CD00011974217530759F416964D915C91179747
:100CE00012962D913C9113974217530769F116966E
:100CF0004D915C91179714962D913C911597215029
:100D000031094217530701F190891696CD91DC9174
:100D10001797988316964D915C91179712962D917F
:100D20003C9113974217530721F42D913C91119751
:100D300006C016962D913C9117972F5F3F4F17963F
:100D40003C932E93169705C0118A128A138A2A980B
:100D500080E0108A1786882321F039C08695808B21
:100D600036C0EF01C453DF4F888199818160998338
:100D70008883DF01A758BF4F14962D913C9115979A
:100D80008D919C9111972817390759F416962D913A
:100D90003C91179712968D919C91139728173907BC
:100DA00061F016962D913C91179714968D919C9118
:100DB000159701972817390751F416968D919C9134
:100DC000179715969C938E9314971982188281A178
:100DD000813618F011A2128A2A98DF91CF911F91C3
:100DE0000F91FF90EF9008951F920F920FB60F9200
:100DF00011242F933F934F935F936F937F938F9320
:100E00009F93AF93BF93EF93FF9380E286BB609174
:100E1000780070917900769567957695679560581A
:100E200080913308909134080E94E204809113016C
:100E3000882349F080913308909134080E94BB03C5
:100E4000807F886001C080E88BB98091FA0490911E
:100E5000FB04A091FC04B091FD040196A11DB11DFD
:100E60008093FA049093FB04A093FC04B093FD04D8
:100E7000FF91EF91BF91AF919F918F917F916F9172
:100E80005F914F913F912F910F900FBE0F901F9048
:100E90001895CF92DF92EF92FF920F931F93CF930B
:100EA000DF931F92CDB7DEB77C01262F82E8860F35
:100EB0008701065E1C4F823010F06B3149F4F80157
:100EC000608171818BE190E029830E94540B29811C
:100ED000D701A05EBC4F3C9111964C911197822F87
:100EE00090E0FC01E327EE0FFF1FE851FF4F259133
:100EF0003491C42ED12C2C253D252D933C93F80103
:100F0000608171810F90DF91CF911F910F91FF90C0
:100F1000EF90DF90CF900C94540BCF93DF93E7E2E8
:100F2000F3E0DC01EF011D922197E9F7FC01E65E99
:100F3000FC4F518340833297718360833A963183AB
:100F4000208332972FEF3FEF318320833297318315
:100F50002083389681E08083DF91CF9108953F927E
:100F60004F925F926F927F928F929F92AF92BF92B9
:100F7000CF92DF92EF92FF920F931F93CF93DF9365
:100F80002C013C0126EE621A2CEF720A6C014BED2B
:100F9000C41A4CEFD40AEC01CC5DDC4F8C01045E2A
:100FA0001C4F7C0182EEE81A8CEFF80A332433944C
:100FB000AA24AA94BA2C4201AEED8A1AACEF9A0A7E
:100FC000F301808191810E94160B8F3FFFEF9F07F5
:100FD00009F459C0F6012081211129C08E379105ED
:100FE000D9F4D8018D919C91429770F0F7018081DE
:100FF0009181883B904F41F42A9AD401ED91FC9164
:10100000309711F0C20109953882F701B182A082B0
:10101000D8011D921C92D4CF8F37910511F41882FC
:10102000CFCF8B31910519F4F6013082C9CF2881D9
:10103000222331F1D8012D913C912831B3E03B07B7
:10104000F0F4A9014F5F5F4FF80151834083F20133
:10105000E20FF31F8083D7012D913C91F901E8271E
:10106000FF27EE0FFF1FE851FF4F85919491232F2B
:10107000332782279327F7019183808301C0188249
:10108000D6011C929DCFDF91CF911F910F91FF90C0
:10109000EF90DF90CF90BF90AF909F908F907F9018
:1010A0006F905F904F903F9008956F927F928F92D4
:1010B0009F92AF92BF92CF92DF92EF92FF920F93E7
:1010C0001F93CF93DF93EC013B014A017C018AED32
:1010D000E81A8CEFF80AF70110825E01F0EEAF1A01
:1010E000FCEFBF0A8FEF9FEFF501918380836E01C4
:1010F000F6EECF1AFCEFDF0AF601608171818EE710
:1011000090E00E94540B8301860C971C081519056A
:1011100039F0F80161918F01CE010E944907F6CFA5
:10112000F501608111816095CE010E944907612F10
:101130006095CE010E944907F601608171818EE7BA
:1011400090E00E94540B81E0F7018083DF91CF9102
:101150001F910F91FF90EF90DF90CF90BF90AF90D5
:101160009F908F907F906F90089590933808809310
:1011700037085093FF044093FE0470933A0860933D
:101180003908109236080895EF92FF920F931F933B
:10119000CF93DF93EC016091FE047091FF0480EC2B
:1011A00090E00E94540B6091FE047091FF0480E077
:1011B00090E00E94540B8E017E0184EEE81A8CEFC1
:1011C000F80AF70120813181225031096091FE0433
:1011D0007091FF04C8018C1B9D0B8217930708F5C3
:1011E000F80181918F01803C59F48BED90E00E94D1
:1011F000540B6091FE047091FF048CED90E00EC0E2
:101200008B3D59F48BED90E00E94540B6091FE04ED
:101210007091FF048DED90E001C090E00E94540BAE
:10122000D0CF80EC90E0DF91CF911F910F91FF9094
:10123000EF900C94540B4F925F926F927F928F922B
:101240009F92AF92BF92EF92FF920F931F93CF9313
:10125000DF93EC018B017A01E0913908F0913A08B3
:101260008289811138C00E94060B90910001891774
:1012700030F4A701B801CE010E94550846C08FB7CF
:10128000F8948090FA049090FB04A090FC04B09035
:10129000FD048FBF209101013091020140910301B3
:1012A00050910401AAE0B0E00E948D0A2FB7F89493
:1012B0004090FA045090FB046090FC047090FD0490
:1012C0002FBF481859086A087B0846165706680653
:1012D000790664F3C1CFE0913908F0913A08818929
:1012E000882309F4B9CF80913708909138080E947B
:1012F000AF07E0913908F0913A08E453FF4F80813D
:101300009181892B41F311821082809136088823C4
:10131000A1F1CA5DDC4F8881811101C0FFCF6091CE
:10132000FE047091FF0480EC90E00E94540B6091E9
:10133000FE047091FF048FE090E00E94540B6091D6
:10134000FE047091FF0481E090E00E94540B6091D4
:10135000FE047091FF0480EC90E0DF91CF911F912B
:101360000F91FF90EF90BF90AF909F908F907F90E4
:101370006F905F904F900C94540BDF91CF911F9121
:101380000F91FF90EF90BF90AF909F908F907F90C4
:101390006F905F904F90089590913B089923A1F032
:1013A000803C01F580910D01811111C010923B0824
:1013B00040913C0850913D0864E171E0809137080C
:1013C000909138080C941B09803C09F086C081E09C
:1013D00080933B088EEF80930D0110923D08109290
:1013E0003C08089520913C0830913D08283193E055
:1013F000390708F072C090910D012115310531F4C3
:101400009E3F21F48F7080930D01089591111FC0AC
:101410008B3D21F481E08093350808959091350843
:10142000992349F08C3D21F08D3D19F48BED01C0DD
:1014300080EC10923508A9014F5F5F4F50933D0833
:1014400040933C08F901EC5EFE4F80830895913093
:1014500079F4282F30E0AAE0B0E00E947E0A609381
:10146000090170930A0180930B0190930C01089578
:10147000943089F42AE0829FC0011124AA2797FDA5
:10148000A095BA2F8093050190930601A0930701C0
:10149000B09308010895933089F42AE0829FC00137
:1014A0001124AA2797FDA095BA2F8093010190934C
:1014B0000201A0930301B09304010895923019F43E
:1014C0008093000108959F3041F4811103C0109270
:1014D0003608089581E08093360808950E949501AA
:1014E0008CE095E00E94AF0780E00E94080288230C
:1014F000B9F30E9412020E94CC09F2CFA29FB00160
:10150000B39FC001A39F700D811D1124911DB29F37
:10151000700D811D1124911D08950E947E0AA59FC2
:10152000900DB49F900DA49F800D911D11240895DE
:10153000A1E21A2EAA1BBB1BFD010DC0AA1FBB1FD7
:10154000EE1FFF1FA217B307E407F50720F0A21B49
:10155000B30BE40BF50B661F771F881F991F1A94B6
:1015600069F760957095809590959B01AC01BD01E0
:10157000CF0108958F929F92AF92BF92CF92DF9248
:10158000EF92FF92CF93DF93EC01688179818A819A
:101590009B81611571058105910521F464E279ED66
:1015A0008BE597E02DE133EF41E050E00E94940B92
:1015B00049015A019B01AC01A7EAB1E40E948D0ADE
:1015C0006B017C01ACEEB4EFA50194010E948F0B7E
:1015D000DC01CB018C0D9D1DAE1DBF1DB7FF03C0EF
:1015E0000197A109B04888839983AA83BB839F7719
:1015F000DF91CF91FF90EF90DF90CF90BF90AF90B1
:101600009F908F9008950E94BA0A08958EE091E00D
:101610000E94BA0A0895A0E0B0E080930E01909372
:101620000F01A0931001B09311010895CF93DF93A0
:10163000EC012B8120FF33C026FF0AC02F7B2B83B8
:101640008E819F8101969F838E838A8190E029C03D
:1016500022FF0FC0E881F9818081992787FD90954D
:10166000009719F420622B831AC03196F983E8831E
:101670000EC0EA85FB85099597FF09C02B8101966D
:1016800011F080E201C080E1822B8B8308C02E81A3
:101690003F812F5F3F4F3F832E83992702C08FEFFB
:1016A0009FEFDF91CF9108950F931F93CF93DF9317
:1016B000FB01238121FD03C08FEF9FEF28C022FF94
:1016C00016C046815781248135814217530744F45F
:1016D000A081B1819D012F5F3F4F318320838C9387
:1016E000268137812F5F3F4F3783268310C0EB0160
:1016F000092F182F0084F185E02D0995892BE1F63B
:101700008E819F8101969F838E83812F902FDF9101
:10171000CF911F910F910895B7FF0C948D0A0E94ED
:101720008D0A821B930B0895052E97FB1EF40094DF
:101730000E94AB0B57FD07D00E94980A07FC03D00C
:101740004EF40C94AB0B50954095309521953F4F3E
:101750004F4F5F4F089590958095709561957F4F9D
:0A1760008F4F9F4F0895F894FFCFBC
:10176A003FC8000000320000005E010000FE0100D8
:02177A0000006D
:00000001FF
